:100000000C942A000C9445000C9445000C94450077
:100010000C9445000C94C0010C94ED010C94150255
:100020000C9445000C9449010C9445000C94450037
:100030000C9445000C9445000C9437030C94450037
:100040000C9445000C9445000C9445000C9445001C
:100050000C94450011241FBECFE5D4E0DEBFCDBF18
:1000600010E0A0E6B0E0EEE3FEE002C005900D92E5
:10007000A43AB107D9F710E0A4EAB0E001C01D929C
:10008000AD3FB107E1F70C94AB000C940000CF93A7
:10009000DF93CDB7DEB7E7E3F0E08FE18083E4E301
:1000A000F0E08CEF8083E1E3F0E084E08083E2E342
:1000B000F0E088E38083DF91CF910895CF93DF93C1
:1000C000CDB7DEB723970FB6F894DEBF0FBECDBF16
:1000D00080E29EE49093FA008093F9001B822FC087
:1000E0008B81482F55278B819927880F991FFC01F9
:1000F000E054FF4F808191819C0128513C4FCA01FF
:10010000880F991FFC01E751FF4F31832083209115
:10011000F9003091FA008B819927880F991FFC0113
:10012000E751FF4F80819181A901481B590BCA01FA
:100130009093FA008093F9008B818F5F8B838B8182
:10014000883070F223960FB6F894DEBF0FBECDBF95
:10015000DF91CF910895CF93DF93CDB7DEB7279787
:100160000FB6F894DEBF0FBECDBF0E9447000E94BD
:1001700027010E9429030E9478031092E70084ED72
:1001800092E09093BB008093BA0082E293E0909358
:10019000BD008093BC0078948091A8008823E1F38F
:1001A0001092A8000E9421060E9460040E94680626
:1001B00000C08091A900813041F41092AA00809182
:1001C000E700882311F40E945E008091A80081302E
:1001D00019F51092A8001A821CC080E690E00E94D7
:1001E000B2038A8199270E94FC0387E690E00E946F
:1001F000B2038A819927880F991FFC01E751FF4FAD
:10020000808191810E94FC030E94ED038A818F5FAF
:100210008A838A81893008F38091A700813049F66A
:100220001092A700C6CFCF93DF93CDB7DEB7F89477
:10023000E9E5F0E089E180837894DF91CF9108953A
:10024000CF93DF93CDB7DEB7DF91CF910895CF93F2
:10025000DF93CDB7DEB7E3E5F0E082E08083EFE443
:10026000F0E01082EEE4F0E082E08083EAE4F0E087
:1002700084EF91E091838083E8E4F0E080ED97E003
:1002800091838083E9E5F0E089E18083DF91CF917C
:1002900008951F920F920FB60F9211242F933F9340
:1002A0004F935F936F937F938F939F93AF93BF937E
:1002B000EF93FF93CF93DF93CDB7DEB78091B1007B
:1002C0008F5F8093B1008091B100883021F40E944B
:1002D00091061092B1008091E6008F5F8093E60056
:1002E0008091E6008834C9F581E08093A9001092DE
:1002F000E6008091B0008F5F8093B0008091B000E5
:10030000853029F41092B00081E08093AA0080919A
:10031000AE008F5F8093AE008091AE00843641F4D2
:100320001092AE0081E08093A60081E08093A80047
:100330008091AE00823319F481E08093A80080910F
:10034000AF008F5F8093AF008091AF008A3029F4B7
:100350001092AF0081E08093A700DF91CF91FF91D1
:10036000EF91BF91AF919F918F917F916F915F912D
:100370004F913F912F910F900FBE0F901F901895A6
:100380001F920F920FB60F9211242F933F934F930A
:100390005F936F937F938F939F93AF93BF93EF93ED
:1003A000FF93CF93DF93CDB7DEB7E091BA00F09122
:1003B000BB000995DF91CF91FF91EF91BF91AF9174
:1003C0009F918F917F916F915F914F913F912F916D
:1003D0000F900FBE0F901F9018951F920F920FB69F
:1003E0000F9211248F93AF93BF93EF93FF93CF930B
:1003F000DF93CDB7DEB7A2E3B0E0E2E3F0E08081C7
:100400008B7F8C93A8E3B0E0E8E3F0E080818F7EFF
:100410008C93DF91CF91FF91EF91BF91AF918F912D
:100420000F900FBE0F901F9018951F920F920FB64E
:100430000F9211242F933F938F939F93AF93BF936A
:10044000EF93FF93CF93DF93CDB7DEB72297DEBF55
:10045000CDBFA2E3B0E0E2E3F0E0808184608C9362
:10046000ECE4F0E011821082A8E4B0E08091A400F6
:100470009927880F991FFC01E751FF4F80819181D7
:1004800011969C938E938091A400882339F4A8E35D
:10049000B0E0E8E3F0E0808180618C938091A4007B
:1004A000282F33273A83298389819A8182309105C5
:1004B000C1F129813A812330310554F489819A812F
:1004C000009789F029813A8121303105D9F04EC059
:1004D00089819A818330910599F129813A8124306B
:1004E0003105E9F143C0A8E3B0E0E8E3F0E0808142
:1004F00080618C93A8E3B0E0E8E3F0E08081816064
:100500008C9334C0A8E3B0E0E8E3F0E080818E7F14
:100510008C93A8E3B0E0E8E3F0E0808182608C9304
:1005200025C0A8E3B0E0E8E3F0E080818D7F8C9304
:10053000A8E3B0E0E8E3F0E0808184608C9316C02B
:10054000A8E3B0E0E8E3F0E080818B7F8C93A8E340
:10055000B0E0E8E3F0E0808188608C9307C0A8E316
:10056000B0E0E8E3F0E08081877F8C938091A40085
:100570008F5F8093A4008091A400893010F01092C6
:10058000A4002296F894DEBFCDBFDF91CF91FF91FA
:10059000EF91BF91AF919F918F913F912F910F90CC
:1005A0000FBE0F901F901895CF93DF93CDB7DEB796
:1005B0008091B2009091B3000097B1F4E6E4F0E0CE
:1005C000808191819093B9008093B800AEE4B0E04F
:1005D000EEE4F0E080818F7B8C9381E090E090935B
:1005E000B3008093B2002BC0E6E4F0E080819181FB
:1005F0009093B7008093B600AEE4B0E0EEE4F0E094
:10060000808180648C932091B6003091B7008091F6
:10061000B8009091B900A901481B590BCA019093E9
:10062000B5008093B4001092B3001092B200809194
:10063000B4009091B5009093FC008093FB00DF9193
:10064000CF910895CF93DF93CDB7DEB7DF91CF91F0
:100650000895CF93DF93CDB7DEB7E7E2F0E01082E5
:10066000E6E2F0E08FEE8083DF91CF9108951F9254
:100670000F920FB60F9211242F933F938F939F9356
:10068000EF93FF93CF93DF93CDB7DEB7E6E2F0E0D1
:1006900010828091A5009927E4E2F0E02081318169
:1006A000880F991FFC01E054FF4F31832083809114
:1006B000A5008F5F8093A5008091A500883010F081
:1006C0001092A500E7E2F0E08091A5008083E6E2C9
:1006D000F0E08FEE8083DF91CF91FF91EF919F91BA
:1006E0008F913F912F910F900FBE0F901F901895F3
:1006F000CF93DF93CDB7DEB7E9E2F0E080E180830E
:10070000E0E4F0E01082EAE2F0E088E18083E0E4F7
:10071000F0E086E88083EBE2F0E082EC8083DF911A
:10072000CF910895CF93DF93CDB7DEB721970FB662
:10073000F894DEBF0FBECDBF8983EBE2F0E080818D
:100740009927807290700097C1F3ECE2F0E0898104
:10075000808321960FB6F894DEBF0FBECDBFDF9128
:10076000CF910895CF93DF93CDB7DEB726970FB61D
:10077000F894DEBF0FBECDBF9E838D838D819E8199
:10078000DC01FD0101900020E9F73197CF018A1BC0
:100790009B0B9C838B831A8219820FC029813A811B
:1007A0008D819E81F901E80FF91F80810E949203DB
:1007B00089819A8101969A83898329813A818B81E3
:1007C0009C818217930750F726960FB6F894DEBFE8
:1007D0000FBECDBFDF91CF910895CF93DF93CDB7FB
:1007E000DEB780916A000E94920380916B000E94A4
:1007F0009203DF91CF910895CF93DF93CDB7DEB70A
:1008000066970FB6F894DEBF0FBECDBF9E8B8D8B63
:100810008D899E894AE050E09E012F5F3F4FB901CC
:100820000E94DA06CE0101960E94B20366960FB6C8
:10083000F894DEBF0FBECDBFDF91CF910895CF9367
:10084000DF93CDB7DEB722970FB6F894DEBF0FBEA9
:10085000CDBF8A8387E089831FC08A81482F5527AF
:100860008981282F332727FD309581E090E0022EE3
:1008700002C0880F991F0A94E2F784239523181663
:10088000190624F481E30E94920303C080E30E94CE
:10089000920389818150898389818823F4F680912C
:1008A0006A000E94920380916B000E94920322963C
:1008B0000FB6F894DEBF0FBECDBFDF91CF91089584
:1008C000CF93DF93CDB7DEB70E94990463E080E059
:1008D0000E94FD058CE690E00E949F0562E081E0A9
:1008E0000E94FD0587E790E00E949F050E948F040B
:1008F000E0E3F0E080819927807290700097C1F763
:100900000E949904DF91CF910895CF93DF93CDB7E3
:10091000DEB78DE00E94D405DF91CF910895CF938B
:10092000DF93CDB7DEB78CE00E94D405DF91CF9185
:100930000895CF93DF93CDB7DEB781E00E94D40551
:10094000DF91CF910895CF93DF93CDB7DEB7269790
:100950000FB6F894DEBF0FBECDBF9E838D838AE0B5
:1009600090E09C838B831CC082E390E09A83898310
:100970000EC08D819E8101979E838D838D819E8186
:100980000097B9F789819A8101979A838983898130
:100990009A81009799F78B819C8101979C838B8327
:1009A0008B819C81009701F726960FB6F894DEBFE5
:1009B0000FBECDBFDF91CF910895CF93DF93CDB719
:1009C000DEB721970FB6F894DEBF0FBECDBF898387
:1009D0008981992781709070882341F0A5E3B0E068
:1009E000E5E3F0E0808180618C9307C0A5E3B0E08F
:1009F000E5E3F0E080818F7E8C9389819927827076
:100A00009070009741F0A5E3B0E0E5E3F0E080816D
:100A100080628C9307C0A5E3B0E0E5E3F0E080815D
:100A20008F7D8C938981992784709070009741F015
:100A3000A5E3B0E0E5E3F0E0808180648C9307C03B
:100A4000A5E3B0E0E5E3F0E080818F7B8C938981C2
:100A5000992788709070009741F0A5E3B0E0E5E336
:100A6000F0E0808180688C9308C0A5E3B0E0E5E306
:100A7000F0E090818FE789238C9321960FB6F8944C
:100A8000DEBF0FBECDBFDF91CF910895CF93DF932F
:100A9000CDB7DEB7A5E3B0E0E5E3F0E080818460A8
:100AA0008C9381E090E00E94A304A5E3B0E0E5E32D
:100AB000F0E080818B7F8C93DF91CF910895CF936D
:100AC000DF93CDB7DEB722970FB6F894DEBF0FBE27
:100AD000CDBF8A838A8182958F70898389810E94A4
:100AE000DD040E9446058A810E94DD040E944605BD
:100AF00022960FB6F894DEBF0FBECDBFDF91CF9127
:100B00000895CF93DF93CDB7DEB721970FB6F89452
:100B1000DEBF0FBECDBF8983A5E3B0E0E5E3F0E023
:100B2000808188608C9389810E945F0521960FB631
:100B3000F894DEBF0FBECDBFDF91CF910895CF9364
:100B4000DF93CDB7DEB724970FB6F894DEBF0FBEA4
:100B5000CDBF9C838B838B819C81DC01FD01019047
:100B60000020E9F73197CF018A1B9B0B8A831982FA
:100B70000EC0898199279C018B819C81F901E80F26
:100B8000F91F80810E94810589818F5F8983998106
:100B90008A81981770F324960FB6F894DEBF0FBEC3
:100BA000CDBFDF91CF910895CF93DF93CDB7DEB75F
:100BB00021970FB6F894DEBF0FBECDBF898381E0C9
:100BC00090E00E94A304A5E3B0E0E5E3F0E08081BB
:100BD000877F8C9389810E945F05A5E3B0E0E5E300
:100BE000F0E0808188608C9321960FB6F894DEBF88
:100BF0000FBECDBFDF91CF910895CF93DF93CDB7D7
:100C0000DEB723970FB6F894DEBF0FBECDBF8A8341
:100C10006B838A81882319F48B81805889838A8128
:100C2000813019F48B818054898389810E94D40595
:100C300023960FB6F894DEBF0FBECDBFDF91CF91E4
:100C40000895CF93DF93CDB7DEB781E090E00E94A7
:100C5000A304A5E3B0E0E5E3F0E08081877F8C9317
:100C600083E00E94DD040E94460585E090E00E943A
:100C7000A30483E00E94DD040E94460581E090E029
:100C80000E94A30483E00E94DD040E94460582E0E6
:100C90000E94DD040E94460581E090E00E94A304CA
:100CA00088E20E94D4058EE00E94D40581E00E9473
:100CB000D40584E890E00E949F056AE081E00E94EC
:100CC000FD0589E890E00E949F05DF91CF9108958E
:100CD000CF93DF93CDB7DEB71092AD000E94990499
:100CE00060E080E00E94FD058EE890E00E949F0594
:100CF00069E080E00E94FD0586E990E00E949F0582
:100D000060E081E00E94FD058DE990E00E949F0572
:100D100060E080E00E94FD050E948504DF91CF9194
:100D20000895CF93DF93CDB7DEB721970FB6F89430
:100D3000DEBF0FBECDBF1982E0E3F0E080819927CE
:100D400080719070009711F081E08983E0E3F0E01A
:100D50008081992788709070009721F0898193E0B5
:100D600089278983998180916900292F281B822FE7
:100D700089838981992787FD909581709070882358
:100D800081F080916900982F8981890F8093690093
:100D90008981982F92708091E800890F815080930B
:100DA000E80021960FB6F894DEBF0FBECDBFDF91ED
:100DB000CF910895FB019F01E8944230C4F0453281
:100DC000B4F44A3029F497FB1EF4909581959F4F17
:100DD000642F77270E940B07805D8A330CF0895DB2
:100DE0008193CB010097A1F716F45DE25193108235
:100DF000C9010C94FB06DC01FC0101900020E9F71D
:100E00003297AE17BF0730F47C91608170833197C1
:100E10006D93F7CF0895AA1BBB1B51E107C0AA1F12
:100E2000BB1FA617B70710F0A61BB70B881F991F8B
:0E0E30005A95A9F780959095BC01CD010895C3
:100E3E004B2000000000003D00010D0A4550492DD9
:100E4E005465737465720056657273696F6E2030E7
:100E5E002E3264006875687500416B6B75005050DA
:100E6E004D2D4F75740050504D2D496E00444D5808
:040E7E002D496E008C
:00000001FF
